S0180000746F7765725F626F6F746C6F616465722E7372656351
S1130000D0F5FF1F11040000EB04000019250000C7
S113001000000000000000000000000000000000DC
S1130020000000000000000000000000EB040000DD
S11300300000000000000000EB040000CD080000F8
S1130040293E0000293E0000293E0000293E000010
S1130050293E0000293E0000293E0000293E000000
S1130060FB350000293E00004D270000293E00001A
S1130070293F0000373F0000E92E0000293E000020
S1130080293E0000293E0000293E0000293E0000D0
S1130090293E0000293E0000293E0000293E0000C0
S11300A0293E0000293E0000293E0000293E0000B0
S11300B0293E0000293E0000293E0000450A0000B8
S11300C0293E0000293E0000293E0000293E000090
S11300D0293E0000293E0000293E0000293E000080
S11300E0293E0000293E0000293E0000293E000070
S11300F0293E0000293E0000293E0000293E000060
S1130400FFFFFFFFFFFFFFFFFFFFFFFFFEFFFFFFF9
S113041072B60E480E49886000220023002400258D
S113042000260027B846B946BA46BB46BC4609482A
S1130430854609488047094880470948804762B68D
S113044000200021074A9047FEE70000000000005A
S113045000ED00E0D0F5FF1F313E00007D200000DC
S1130460B52000007B1A000000000000000000001E
S1130470002A01D101207047F0B41F46034603242B
S11304802340002B09D00424E31A0170013008240E
S1130490E141521E26D05B1EF7D1042A1ADB13D089
S11304A0002F11D00C460D460E46102A02DB72C0F6
S11304B0103AFAE70C2A02DB32C00C3AFAE7082AAF
S11304C002DB12C0083AFAE7042A03DB01600430B5
S11304D0121FF9E7002A05D0017001300824E14118
S11304E0521EF7D1F0BC00207047FEE7E510000073
S11304F000000000F7100000000000006B11000075
S1130500691200004B110000BF11000045130000E8
S113051000000000D11300000000000009110000D9
S11305200000000000000000000000006113000053
S1130530000000000000000000000000A710000000
S1130540000000003711000000000000000000005F
S11305500000000000000000000000000000000097
S11305600000000000000000000000000000000087
S1130570000000000000000000000000000102462E
S1130580BD1A0000811B0000000000009D1B00003C
S1130590391C0000D91C00000D1D0000631D000063
S11305A0751D0000051E0000391F0000000000003A
S11305B0000000000000000000000000291B0000F3
S11305C0991E000000000000000000000000000070
S11305D00000000000000000F5400000FF400000A3
S11305E0094100000000000000000000F92500009F
S11305F0452600009D2600000000000000000000C9
S1130600D12600003515000065150000A91500006D
S11306109916000000000000D5160000BB29000058
S1130620AF2B0000CF2B00000000000000000000F2
S1130630012C00005B360000A5360000593700008D
S11306400000000000000000953700003524000081
S11306509D220000C92200005923000095230000B8
S11306601523000069220000712200007D22000091
S11306708D220000000000000000000001000000C6
S1130680000000005B09000024070000340700009C
S11306900807000002000000000000009D0900009F
S11306A034060000440600000807000004000000AF
S11306B000000000CD090000EC050000FC0500006E
S11306C0080700000800000000000000150A0000F0
S11306D01C0600002C0600000807000000000000B3
S11306E00000000000000000000000000000000006
S11306F000000000C1370000FB370000193900007A
S1130700D539000078F2FF1F713A00007D3A0000ED
S1130710ED3A0000A33B0000753A0000AF3B000037
S1130720513A0000513E0000CB3E0000E53E00007F
S11307300000000000000000133F000038B5050071
S1130740414C002323620020002103C4083C220002
S1130750083203C22200103203C263623B4800F035
S1130760A6F8183403C43A49280000F07DF931BDD5
S113077070B50C00344D296A07291CD1696A884276
S113078019D100F0A0F89626F60001010A1A03CD4B
S1130790030003CD1918100000F0A6F90A214843FC
S11307A0310000F0A1F9401D0A2100F09DF97043C9
S11307B02060002070BD012070BDF1B582B000F052
S11307C066F804000D00204E376A7F1C3000183094
S11307D003C8009001913000103003C82B00221A86
S11307E08B4100980199994203D801D3904200D2D9
S11307F001273762012F06D0042F09D0052F0FD00F
S1130800072F11D01CE030C6083E0298706217E032
S11308100CCE083E2900A01A994103C6083E0FE0F9
S11308203000083030C00BE0300008300CC829001C
S1130830A01A99413200083203C2029800F028F944
S1130840103630C6F7BD000008F1FF1F80380100E4
S1130850BB07000010B5204C002020601F49204A2F
S11308604A608860072008601E480068C0001E496E
S113087000F03AF9002800D10120606010BD17484B
S11308800168072291430160002181607047124989
S11308900A6816480068C3431802000A0B689A42A3
S11308A0F6D1130A1206002180185941704700B589
S11308B00021094A5268002300F032F9C0084A07AF
S11308C01043C90800BD0748006870470248016822
S11308D0491C0160704700006CF2FF1F10E000E04B
S11308E0FFFFFF0000F1FF1F40420F0018E000E08F
S11308F010B58207D30EFF249C40E2438907090EFA
S11309009940030004D56D481B071B0F083B00E00A
S11309106B489B089B00C01803681A401143016090
S113092010BD890040180168664B0B401104F02289
S113093012030A401A430260704789004158C801F3
S1130940C00F704700E000BF1202E023DB00134039
S1130950890043507047F7E7F6E7002800D0704756
S113096010B5594C002903D002290CD003D310BD73
S11309702064606410BDA00D206454480168544A8A
S11309800A40026010BD032210212000FFF7DAFFA5
S1130990032211212000FFF7D5FF10BD002800D04D
S11309A0704710B5484C002902D0022903D010BD6D
S11309B02060606010BD022201212000FFF7C3FF08
S11309C0022200212000FFF7BEFF10BD002800D046
S11309D0704710B53F4C002902D0022905D010BD44
S11309E020646064A064E06410BD02221021200031
S11309F0FFF7B1FF022211212000FFF7ACFF022212
S1130A0012212000FFF7A7FF022213212000FFF785
S1130A10A2FF10BD002800D0704710B52D4C00294E
S1130A2002D0022903D010BD6066206610BD0222E8
S1130A3019212000FFF790FF022218212000FFF760
S1130A408BFF10BD80B510211F48FFF776FF0028EB
S1130A5009D021480168080005D0002088470020FB
S1130A60C0431E49086001BD10B50C0000280ED11A
S1130A7001211F20FFF73CFF802000061849086071
S1130A800A2210211048FFF74CFF1348046010BDE0
S1130A90002800D0704780B5802000061149086006
S1130AA000211F20FFF724FF002210210648FFF732
S1130AB038FF00200849086001BD00001CED00E07B
S1130AC000E400E0FFFFF0FF00A0044054F00F40FA
S1130AD0FFFFFEFF00D0044074F2FF1FA0A00440FB
S1130AE000E100E080E100E0094214D088420FD325
S1130AF00122030C01D100041204002300185B41FD
S1130B008B4200D35B1A5241F8D31900100070478E
S1130B1001000020704708B500F01CF808BD000073
S1130B2030B4434351435D18010C0C00130C5C4377
S1130B302D1980B2434392B251430024C918644131
S1130B4024040B04090C09195043C018694130BC32
S1130B5070470000704700000021C943C26E8A42FA
S1130B6005D1026F8A4202D1426F8A4201D02B49D9
S1130B7000E02B49C16270473EB504000D00684691
S1130B8000F05AF820000C302818001B051DA2683C
S1130B906168A9420BD28B18984208D2421A68465F
S1130BA000F050F86068A1684018421B29006846AC
S1130BB000F048F802A9684600F06FF802983EBDBC
S1130BC058B50126174881680C69E16A144A9142B4
S1130BD021D00026220068329168002919D0526879
S1130BE04B42934215D3406803689A4211D340683C
S1130BF05118491E88420CD30B4920006830FFF776
S1130C00BBFF616F884201D0084803E00126084811
S1130C1000E00848E062300052BD0000A228000055
S1130C20A328000010F0FF1FC0A30000A1280000AB
S1130C30A0280000A42800000021C943016000216D
S1130C4041607047F0B585B004000E001700684697
S1130C5000F092F868460121C172216801911B4994
S1130C600091002181720181002F0FD000F01CF946
S1130C70174D6946280000F04DF83A00310028006D
S1130C8000F081F82868019000F014F901982060C0
S1130C906068C019606005B0F0BD38B504000D008F
S1130CA020798007800F08D0694600220A60042159
S1130CB00A1A69462000FFF7C5FF20682860054826
S1130CC00168054A0A40026031BD0000B71DC10435
S1130CD0002003403C800440FFFFFBFF10B54A7A2C
S1130CE092070B7A1B07C024A4051C4014438A7A7C
S1130CF093062343CA7A12068024640422401A43CA
S1130D0082600B6843606300134383604968016039
S1130D10826010BD70B584B0164A13688024E40262
S1130D201C4314600322022300240D7B002D0D6854
S1130D3000954D6801956D460DD14E7A002E01D077
S1130D402B7200E02C720C7A002C00D002226A7202
S1130D508A7AAA7207E02C720E7A002E01D06B7286
S1130D6000E06A72AC72C97AE9726946FFF7B6FFAD
S1130D707FBD00003C80044080B500BF13A1102259
S1130D8000F0BAF801BD03E00B780370491C521E51
S1130D90002A06D08B07F7D103E00B680360091D16
S1130DA0121F042AF9D2002A03E00B780370491CAD
S1130DB0521EFAD17047016880688000800F0228B3
S1130DC001D3080C704788B270470000211000005E
S1130DD0FFFF0000000000000000000070B50400E8
S1130DE00E00394D03CD083D002906D1002804D159
S1130DF0FA208000FFF75BFD03C566700023002026
S1130E00207000212200083203C2236170BD70B536
S1130E1004000E0000256078002807D072B66078C0
S1130E20401E6070257062B6002070BD002E13D085
S1130E302078002812D0FFF72AFD220008320CCABD
S1130E40801A9941204A0CCA00F070F82169814245
S1130E5012D272B6257062B6022070BD0020C04363
S1130E60864209D072B60120207062B6FFF70FFDEA
S1130E702200083203C22661032070BD4178FF2995
S1130E8001D10120704772B64178491C417062B6A5
S1130E90002070470021016062B6704772B60020DE
S1130EA00A49086062B6704772B608480168491C6E
S1130EB00160704705480168022900D2EAE7016829
S1130EC0491E01607047000088F1FF1F64F2FF1F94
S1130ED0124207D08B0706D00B78491C0370401CC4
S1130EE0521EF7D87047830706D00B78491C03704D
S1130EF0401C521EF9D1704770B4103A03D378C91C
S1130F00103A78C0FBD2530701D318C918C001D5D1
S1130F1008C908C0D20704D30B880380891C801C2D
S1130F20002A01D50B78037070BC7047124224D09C
S1130F30994228D970B500251B4202D00C0000212B
S1130F4009E00024012649186441944200D3A41AFC
S1130F507641F8D33100012601E0764109D2001828
S1130F6064416D41A41A9D41F7D2A4185D41B6199C
S1130F70F5D3300022002B0070BD1B42D8D108B538
S1130F80FFF7E8FD08BD01D19042D3D202000B0067
S1130F9000210020704700000020B049C968C968DA
S1130FA008607047FEB5002600206A469670AB4C78
S1130FB0E7697D69002D75D0E168C9680A68012A6E
S1130FC05AD000230A000832091D38006D68A8476A
S1130FD0002805D0A249884202D0491C884261D128
S1130FE0E268D1688B68002B5CD00293486801905A
S1130FF000786B46187068460078002808D0684668
S11310000078132804DA9268C0001018083800E049
S1131010002008620127002822D0006800281FD081
S113102000A9491C200020302269926990470500DC
S113103017D168464078002809D0E7204001694666
S11310400978491EC840384001D1864D09E002990B
S11310500198E268D268126A12689047002007E09B
S1131060B74D68460178280000F0BCF9280019D172
S1131070E168C9680F60FEBD096A00290DD049689E
S1131080080003D000A8801C884700E00020002846
S113109003D0E168C9680E60FEBD69468978E268DC
S11310A0D2681160FEBD80B50178002000F09AF985
S11310B06A48C069416909698847022000F0D6F985
S11310C0BFF34F8FA448A5490860BFF34F8F00BFFB
S11310D0FDE780B514216148C068C0680C3000F099
S11310E021FA01BD10B5040000F01EFBFFE72178D2
S11310F000F078F910BD10B50400A1686068574A83
S1131100126852699047F2E77CB500240194009478
S1131110524D6B4601AA8168C9B24068C0B2AE683C
S1131120B668B047E968C9680C6100998A080199F2
S113113000F060F973BD10B50400A1686068C0B226
S1131140464A9268D2689047D1E710B50400FFF789
S1131150C0FF4248C068C068A1680161616841611C
S11311600421017721780020C2E710B50400FFF7BD
S1131170B0FF3A48C068C068A16801616168416114
S113118003210177A168002000F048F910BD38B5AB
S11311900400324DE868C068002141610161007FAC
S11311A0042805D1286800698047002C00D1040078
S11311B0E868C068017F200000F014F931BDF1B582
S11311C084B0264DE868C06800240169002905D16F
S11311D0049804700020FFF7DAFF3CE00121049A30
S11311E011700769406901900094E86901236A4617
S11311F002A946697668B047060004D0E8694169E7
S1131200C96888471CE00098002801D1144818E0F8
S1131210B84200D938000090029A014601982B6820
S11312209B6898470600019800994018019000981F
S11312303F1A05D0002E09D0E8694169C96888477A
S11312403000FFF7A4FF0498047004E0E868C06865
S1131250076101994161002005B0F0BD10F0FF1F46
S11312601227000011270000F1B58CB07D4FF868FB
S1131270C06800250169002905D10C98057000207B
S1131280FFF785FF59E001210C9A11700169029161
S11312904469C168027F029B212B00D32023019360
S11312A0002915D0019A04A8FFF712FE02980199AB
S11312B0401A0290F8690123019A04A94669B668A4
S11312C0B0470600029800282CD0002E30D029E028
S11312D0019961180391032A07D104AA01992000F6
S11312E03B685B689847060012E0102A01D00C4660
S11312F0DCE7467FFFF7D8FD0096019B04AA210096
S1131300380020303C69E46BA0470600FFF7D2FDAB
S1131310039C002ECAD0F8690123002204A9446961
S1131320A468A0473000FFF732FF0C98057004E072
S1131330F868C06802990161446100200DB0F0BDF5
S11313401027000010B50400E268A1686068454BEE
S11313501B68DB689847CAE60400FA050CED00E058
S11313607CB5060070680090B0680190F0683E4C4F
S1131370206000253B4949681031002807D00A68DD
S1131380904203D34968491C814200D20425009845
S113139000F08EFA002800D104253178280000F0EE
S11313A021F8002D13D100986060002000F05EF851
S11313B00198A0602068002803D080F3088880F397
S11313C00988A06861688847002000F04FF873BD61
S11313D010B50400234A211D100020301269D2697F
S11313E0904784E610B584B06A46A02313700023A6
S11313F0537028E030B589B06C46A72323700023CE
S11314006370A370551CE570019004E098000D58BA
S1131410201885605B1C9342F8D304E010B584B0B7
S11314206A46A3230BE00F48C0690023E1788A00D1
S1131430121D69464469A468A04709B030BD137001
S113144001235370002393700223D37001900291FF
S11314500448C06900230C2269464469A468A04773
S11314601FBD000010F0FF1FB4F1FF1F70B5050091
S11314700024022D04D0002000F0A6FD012D0ED082
S1131480002605E0C16889680A0000D08847761CF8
S11314900D4818217143401801680029F2D1002D2C
S11314A00DD1FFF701FDFFF7EAF900F003FE07484D
S11314B00460012000F01EFE00F07CFE62B6BFF363
S11314C06F8FBFF34F8F70BD7C06000008ED00E006
S11314D0094205D083070BD00270401C491EF9D184
S11314E0704700001206130A1A43130C1A4300BF74
S11314F0130030B414001500103902D310393CC065
S1131500FCD2490700D30CC000D504C0890002D323
S11315100280801C002900D5027030BC7047000096
S11315200022D5E70022E3E7EFF31080BB494860CF
S113153072B6704738B5BA4C65682A000421200099
S113154020302369DB6A98476A4601212000203055
S11315502369DB6A9847286800994018401E686030
S1131560002032BDF8B504000D001600C14F796BA0
S1131570484201002140621A521953421840424223
S11315806B46380020303F697F6CB84700280AD189
S113159068460078002801D06C20F2BD3200290092
S11315A0200000F065FEF2BDF5B58BB00D0003AA76
S11315B000F038F904006AD1A808800004902F1ABA
S11315C00020C04308900990002F06D03A000C98E0
S11315D00499411808A8FFF77BFCFFF7A5FF0B98B7
S11315E00499401807908E4D0498002809D00346AA
S11315F00C9A0B99280020302C696469A0470400D8
S11316000AD1002F08D0042308AA07992800203003
S11316102C696469A0470400804E706880F31088C8
S1131620002C34D16846007B002832D0FFF77CFFC1
S11316300498002812D005A8029006A80190A86872
S11316400069006DC0B200900C9B049A0B992800AD
S113165020302C69A46AA047040013D1002F11D0B4
S113166005A8029006A80190A8680069006DC0B2A0
S1131670009008AB08220799280020302C69A46A3E
S1131680A0470400706880F31088002C01D020006B
S113169000E000200DB0F0BD70B588B005000C006E
S11316A0002069468300CA50401C0828FAD3002C45
S11316B00DD02026202C00D826006A4631002800B0
S11316C0FFF772FF002803D1AD19A41BEFE7002038
S11316D008B070BDF8B507000E00FFF725FF504CA9
S11316E0654B320039002000203025692D69A84758
S11316F04A4D696881F31088002814D1A1680969EA
S1131700096B00290FD0FFF70FFFA0680069036D74
S1131710DBB232003900200020302469646AA0471B
S1131720696881F31088F2BDF8B500203C4CA168CB
S113173009690D0058358A696768296856423A680C
S1131740914228D1696891422ED1FFF7EDFE4A49B2
S113175020002030226992689047304D696881F3F7
S11317601088002816D1A1680969096B00290FD0D7
S1131770FFF7DAFEA0680069016DC9B220002030CD
S11317802269126A9047696881F31088002801D1A0
S113179001212970F2BD8A4206D2314004D01000E2
S11317A0FFF798FF0028F5D169684A421640724253
S11317B079688A42EED2491C891A1000FFF78AFF21
S11317C0F2BD70B582B0150000222A70144C6B462D
S11317D00A000100200020302669766CB0470028FA
S11317E019D169460978297069460978002912D007
S11317F00A4D297800290ED1A0680069016DC9B28B
S1131800200020302269126A9047002801D06C2001
S113181076BD0121297076BD000000004CF2FF1F47
S113182010F0FF1F70B582B005000E0014001148BF
S113183080680069006B002800D001202070FFF749
S113184073FE6A4670420321884341422800FFF731
S1131850B8FF0A494968002802D081F3108876BD90
S113186081F3108868460078002801D00020207099
S1131870002076BD10F0FF1F6B66656B4CF2FF1FF6
S113188038B505000C000020FFF7F0FD8248046025
S11318904560A0210902814A1160016881F308882A
S11318A081F30988406880470020FFF7DFFD31BDE0
S11318B010B582B0002806D00021C943884202D066
S11318C07749884201D1002016BD00246A460221CE
S11318D000F06DFD002804D10098007A002800D0A3
S11318E00124200016BDF0B589B06E4EB0680069C1
S11318F0683001906C4F3D000AE00199097C014277
S113190005D0686981692800EA68526890471835EB
S113191028680028F1D1002104AA03C202AA03C244
S1131920FA208000FEF7C3FF06AA03C208210020A4
S113193000F094FD002805D1A02000024168009128
S1131940046801E00024009400F054FC00283AD11B
S11319500098FFF7ADFF002835D0FFF731F90028D4
S113196031D0B068006986300078C00703D4210004
S11319700098FFF785FF0198408A4C49884200D1BE
S11319804B4802AD002106AA0CCAFFF7C9F803C5EB
S1131990FEF77DFF04AA03C202A803C8002901D1EF
S11319A0002810D0FEF773FF04AA0CCA801A9941CC
S11319B002AA0CCA994206D301D8904203D321004B
S11319C00098FFF75DFF3D0000E018352868002807
S11319D0E2D00199097C0142F7D02800E96809683E
S11319E088470028F1D0002DD6D00AE00199097C5F
S11319F0014205D0BD4203D03800F96889688847A0
S1131A00183738680028F1D1280009B0F0BD10B5A6
S1131A10FFF744FA00F0C4FB224C20002030216977
S1131A20496888472348E063200020302169096C15
S1131A308847A06800688047002000F05BFBFEF741
S1131A4009FF206800688047A06840688047FFF766
S1131A504AFFE0610169002903D009680A0000D047
S1131A608847E0694169002903D009680A0000D069
S1131A708847E0680068804710BD38B5FFF7C7FFA6
S1131A80084CE569E06840688047E868C168080078
S1131A90F8D028008847F5E7C0F1FF1F08ED00E003
S1131AA01104000010F0FF1F7C060000FFFF00007F
S1131AB08813000064F0FF1F7047000010B5002871
S1131AC001D1042010BD7F4909680901090F0F29BC
S1131AD002D18022920203E00BA24900515A8A02E9
S1131AE000210160426001228260D202C260764A13
S1131AF0930D1478A3404361D2788261016101623D
S1131B004162002010BD00000800100018002000F1
S1131B103000400060008000C0000001800100022D
S1131B20000300040006000070B5002801D1042061
S1131B3070BDC46965680C2209A12800FFF7C8F9C3
S1131B40624E6D1C3560A568142200BF07A12800F1
S1131B50FFF7BEF96D1C756002202060002070BD87
S1131B608021017002780A42FCD07047016880220B
S1131B70D2000A430260BFF36F8FBFF34F8F7047E9
S1131B8038B5040001D1042032BD5148514A1060D7
S1131B905D48814201D06B2032BD44E0F8B58AB083
S1131BA007000C00150001AA00F049FA059B2A0061
S1131BB02100380000F02CFA060023D1019C029881
S1131BC0009065196D1E28000099FEF78DFF00290D
S1131BD00AD028000099FEF787FF451C009845436A
S1131BE06D1E01E000982418A54218D32002000AB3
S1131BF0902109050143374801600A984249884207
S1131C0003D06B2630000BB0F0BD380000F0BEF9F5
S1131C1006003869010000D08047002EE2D0380069
S1131C2000F0D2F9EEE7200000F0B0F90500200042
S1131C3000F0CAF9280032BDF1B588B00D001400D7
S1131C401F00002C01D1042039E06A4600F0F7F9A6
S1131C50039B3A002900089800F0DAF906002ED117
S1131C60009D02E003982D183F1A002F23D020680E
S1131C7018494860241D03992802000A042905D143
S1131C80C021C90401431348016009E0082907D1B0
S1131C902168104A9160241DE021C90401431160A8
S1131CA0089800F073F9060008980069010000D054
S1131CB08047002ED6D0089800F086F9300009B08D
S1131CC0F0BD00004C800440280002405CF2FF1F7D
S1131CD0FFFFFF4404000240002801D0002901D185
S1131CE0042070476A4800788207920F022A01D1C3
S1131CF0002006E0C0220240802A01D1012000E039
S1131D0002200870002070476B66656B10B50200F6
S1131D1001D0002901D1042010BD00205C4B1C78A7
S1131D20A407A40F022C1BD05A489B1C18600878E7
S1131D3000064C7824040443887800022043CC78BD
S1131D4004435C60087900064C79240404438879D0
S1131D5000022043C97901439960100000F016F98C
S1131D6010BD80B5002801D1042002BD0904714AC8
S1131D7084E00000F9B589B00C00160001AA00F057
S1131D805EF9069B32002100099800F041F9002811
S1131D9036D101AA2100099800F051F9019C039859
S1131DA00090604200994A4202405542A54205D142
S1131DB06D1803E0F61BE41900982D18002E1ED0B0
S1131DC0281B3700864200D9070038000699FEF721
S1131DD08BFE2102090A802252040A436A490A60DE
S1131DE00AA90978090200040843FF21014366484F
S1131DF04160099800F0CAF80028DBD000E0002018
S1131E000BB0F0BDF1B588B00C0016001D0001D177
S1131E10042031E06A4600F012F9079B32002100E9
S1131E20089800F0F5F8002826D1009C564F05E0EC
S1131E300799761A8A089200AD186418002E1BD0F0
S1131E402002000A80218904014339600EA8007829
S1131E5000060E49014379602868B860089800F0CC
S1131E6095F80028E4D00F99002900D00C6010994F
S1131E70002901D000220A6009B0F0BD0A4351498B
S1131E800A6000F083F802BD00000000FFFFFF00BD
S1131E9002000240FFFFFF45F9B585B00C001500B4
S1131EA0002B01D1042043E0042300F0B1F8029098
S1131EB000283CD10026002760190190059840694C
S1131EC000900146484201994A4202405142204052
S1131ED0081A0099FEF708FE0390012509E041491C
S1131EE009682038CA43C2402A4000D07F1C0098A9
S1131EF02418019884420CD220000099FEF7F4FDC6
S1131F00202802D237494968ECE705998969884253
S1131F10E5D3002F02D10698067008E003988742A3
S1131F2003D202200699087001E006980570029811
S1131F3007B0F0BDFFFF0040002801D0002A01D106
S1131F400420704709291CD801A35B5C9F4400BF8F
S1131F500A1212161A1E22262A2EC06810600020A9
S1131F6070474068FAE78068F8E70068F6E7012000
S1131F70F4E74069F2E78069F0E7006AEEE7406A57
S1131F80ECE76A20704700000400024010B5164CCC
S1131F907021217000F02EF8002811D1200013497F
S1131FA0096888472078810601D5672010BDC106DD
S1131FB001D5682010BDC00701D5692010BD0020DF
S1131FC010BD00000400024038B50400200000F0F9
S1131FD011F80500002D03D10548044949688847D4
S1131FE031BD000018000240000002405CF2FF1FF7
S1131FF00C3000F0002801D104207047C06900288B
S113200004D00068022801D1002070476D20704779
S1132010002801D1042070475B1E194201D11340EE
S113202001D0652070470368994204D340681818AA
S11320308918884201D2662070470020704770B525
S113204005000E001400002D01D1042070BD2021D4
S11320502000FFF767FA2868301A2060E86860609B
S11320606868A968FEF740FDA0600420E0600821CC
S113207021616161A061E061002070BD80B51148FB
S11320801149086011491248421A1248884203D083
S1132090002A01D0FEF71CFF0F481049091A01D08D
S11320A0FFF73EFA0E490F48421A02D00E48FEF7D7
S11320B00FFF01BD0020C0430C4908600C490860B3
S11320C0704700000000000008ED00E0A83F000099
S11320D0AC40000000F0FF1F08F1FF1FD0F3FF1F0A
S11320E07041000070410000D0F3FF1F80E100E068
S11320F080E200E0F8B52449244C00283ED1206851
S113210008602348806800696830A0277F04017F45
S1132110C90708D521683800090F491CFEF7E4FCFB
S11321201C490860F1BD407FC1430D072D0F6D1C94
S113213038002900FEF7D8FC060017488642F6D27C
S113214020684003470F7F1C009600E07F1C304648
S11321503900FEF7C9FC11498842F7D2012D01D19B
S1132160092F0FD26D1E28077F1E3904E022D202E8
S11321700A400243226007480660F1BD012801D1EC
S113218008682060F1BD00BF48F2FF1F448004408E
S113219010F0FF1F00F1FF1FC168780441787D0132
S11321A080B500F071F928480168F82292010A43C9
S11321B0026001BD24480168244A0A400260704755
S11321C000B523480168234800684903490FFFE725
S11321D0491CFEF789FC00BD80B5002802D0012807
S11321E003D005E01B48006802BDFFF7E9FF02BD0C
S11321F0002002BD10B51849880D086017484268D0
S113220080239A4342600A68132313430B6000211E
S1132210FA22520003681C06E40F0919521EF9D170
S1132220FA298041C00F10BD0D480068000E000758
S113223008D10C48806800697821415CF7220A4083
S1132240783002707047000038800440FFC1FFFFFF
S11322504480044000F1FF1F1CB0044090F00F4084
S11322602480044010F0FF1F80B500F025F902BD62
S113227080B513000A000100180003E080B51300C4
S11322800A001900FEF724FE002002BD10B50C0060
S1132290110001232200FEF7EBF810BD70B582B0E7
S11322A004000E001500002E01D1002076BD6A4600
S11322B000F07DF8002806D12A0031002000009BA0
S11322C0DB685B68984776BD70B582B004000E0089
S11322D01500002E01D1002076BD00F08DF80028F5
S11322E001D05B4876BD6A463100200000F05FF8FB
S11322F000280ED12A0031002000009BDB689B6877
S113230098475449002802D1009AD26800E000227C
S11323100A6076BD38B504000D006A4600F047F83F
S1132320002815D10098C0684069002801D16620B2
S113233032BD2900200000F05FF8002801D0444895
S113234032BD29002000009AD2685269904732BDFC
S1132350002DFCD1002032BD70B582B004000E0007
S11323601500002E01D1002076BD00F045F80028AC
S113237001D0374876BD6A463100200000F017F8D6
S1132380002806D12A0031002000009BDB68DB68AE
S1132390984776BD38B5002400202E4D29680029C1
S11323A004D009690A0001D088472C6032BD0300BB
S11323B02748002A00D1704770B5274C6468146020
S11323C0002902D170BD103414601468002C12D09E
S11323D02568002D05D16668002E02D1E668002E1E
S11323E009D0AB42EFD365689D42ECD35918491E1E
S11323F08D4200D3002070BD70B54118491E0022E3
S1132400154B9C682469D500641958345D6816011D
S1132410AD5966682468AC4201D1AE4205D086420B
S113242003D3A14201D3012070BD521C022AE8D378
S1132430002070BD10B50848446804E0006801003D
S113244000D080471034E0680028F7D110BD0000A8
S1132450D827000068F2FF1F10F0FF1F10B582B0EC
S113246000226B461A70074C0A000100200020303D
S11324702469646CA04768460078002800D00120D5
S113248016BD000010F0FF1F0948817804290DD102
S113249001789F220A400270FF218278012A03D129
S11324A0044A1278520701D4491EF6D1704700003D
S11324B001E0074002D007400C4800680003010F08
S11324C0082910D2802292008A400CD00848406823
S11324D01030910880229205521A02604A00511865
S11324E0044A891841600020704700BF24800440DA
S11324F010F0FF1FFFFFFF1F002807D18020C0003E
S1132500012901D1024900E002490860704700BF77
S113251000E100E080E100E0BFF34F8F034804498D
S11325200860BFF34F8F00BFFDE700BF0400FA054A
S11325300CED00E0002807D180204000012901D1E2
S1132540024900E002490860704700BF00E100E072
S113255080E100E001280CD8012200BF07A3185C29
S1132560C006C00E8240012901D1024800E00248A1
S11325700260704700E100E080E100E00C0D000023
S1132580002101807047F0B585B005000E001700EA
S11325906846FEF7F1FB00206946C8722A8801925A
S11325A0114A009288720881002F11D0FEF77CFC3A
S11325B00E4C69462000FEF7ADFB3A0031002000C6
S11325C0FEF7E1FB2000FEF7F6FB0190FEF772FC3C
S11325D00198288005B0F0BD00880880044801688F
S11325E0044A0A40026070472110000000200340A2
S11325F03C800440FFFFFBFF4F494068085C704784
S11326004D498A68002A08D04A6813780370521C1E
S11326104A608868401E88607047002101707047D6
S11326205A2800D0704780B5434A01235354434984
S113263011615169884701BD80B53F49496988479F
S113264001BD0000F0B585B004003B4D696100BFD9
S113265041A0616889004758684600F0E8F80126FF
S11326606846067246723648E86036482861022198
S11326706068A26890476946380000F08BF83249D8
S1132680380000F013F901216068FFF735FF606836
S113269028184670002005B0F0BD000070B5040095
S11326A06068254D29184978002910D02AA1820094
S11326B08E580021FFF720FF300000F0C3F80021FE
S11326C06068A2689047002061686918487070BD0E
S11326D019484160826081680029FCD1002070475C
S11326E0F0B583B0070000BF1BA0B90040580090AC
S11326F004462C34206880210905084009D0216053
S113270007E001A8E96888476846007900994863AA
S113271026602068084D8026B6043040F1D1206838
S1132720310A084007D00098806B21603900C0B29C
S11327302A699047F3E7F7BD70F0FF1F39260000C0
S113274001260000212600000000020A80B50020B6
S1132750FFF7C6FF01BD000000C00240010C4E4A55
S113276089180A680123834013430B6070470029CA
S1132770016802D0494A0A4002E08022D2010A4399
S11327800260704701000020454A914200D00120B8
S11327907047000038B505000C00FFF7F3FF00BFD9
S11327A035A180000858FFF7D9FF01212800FFF761
S11327B0DEFF2868012101432960286840004008A1
S11327C02860286837490140207B80070843A17BA3
S11327D089060143607B00060843E17B0902C022AD
S11327E092000A4002432A6001220121280000F0DD
S11327F045F8207880002818C1682B4A0A4061688F
S1132800491ECB06F021C90519401143227A9206CC
S11328108023DB041A400A43617A49065B081940A5
S11328201143C160286801218843286031BD00211B
S11328300170082242600172417201734173817315
S1132840C173704738B50500012428682043286007
S113285000212800FFF78BFF2800FFF793FF00BF3C
S113286005A180000858010C0B4A89180A688440A5
S1132870A2430A6031BD00000C003C1010B503688F
S11328800C04F82149032140012A02D119430B0009
S113289000E08B43036010BD00700440FFBFFFFFE6
S11328A000C00240FFCCFFBAFFFFFF808A0103D5BE
S11328B0026B064B134003638A0303D5026B044B7C
S11328C013400363026B114301637047FFFFFFFE74
S11328D0FFFFFEFF8021890402680A430260026848
S11328E00A40FCD170470168404A0A40026001680E
S11328F0C14A0A4002600168C901FCD470470168FA
S11329008022D2050A4302600168802252050A43EC
S113291002600168C901FCD5704738B505000C0098
S1132920032C02D1FFF7EBFF06E0042C04D1286846
S113293080210906014329602800FFF7E0FF002CED
S113294004D12868AD49014029600BE0012C02D173
S11329506868082104E0022C04D1686880214901D8
S11329600143696025E038B505000C00032C02D151
S1132970FFF7B9FF05E0042C03D1286840004008A4
S113298028602800FFF7BBFF002C05D128688021B0
S11329900904014329600CE0012C04D16868082172
S11329A08843686005E0022C03D16868AA490140A5
S11329B069602800FFF797FF31BDA84940680818EF
S11329C0407870475A2800D0704780B5A34A012345
S11329D051184B70A249A34B59655168884701BDF2
S11329E080B59E494968884701BD0000FFFFFFEF9D
S11329F0F1B58AB09C480A9989004058069001A80C
S1132A0000F084FB012401A804711021417197484E
S1132A1080680069030094331F88924D2E00383675
S1132A209349944A974201D00F4001E0FF2724378D
S1132A30B7825B88934201D0194000E08E49F1824D
S1132A409130007800270107090F0F2901D1B474D0
S1132A5023E0B77401071BD50521317483498968C4
S1132A60096992310988009107A9009A12120A7023
S1132A70009A1206520F8A70009AD206520FCA7038
S1132A80009A9207920F4A704006400F087106E0C0
S1132A904007400F3074052801DB04203074AD4832
S1132AA0F06110203056002803D0022806D002D34B
S1132AB006E0A94805E0FA20800202E0A74800E009
S1132AC0A7480190002128000830FEF787F900216B
S1132AD028002030FEF782F9082028600920686069
S1132AE0069DA04A01A9280000F08AFA2968490035
S1132AF0490829602968C902FCD46868A103014314
S1132B00696010203056052806D10420307407A9C6
S1132B10280000F006FB06E0954982001018091809
S1132B20280000F0FEFAB07C002804D0747401215F
S1132B302800FFF7F2FE37700820706004A80771C0
S1132B40F18A89048B4A0A4004924771012304AA3A
S1132B500821280000F033FBA86A21020143A9627E
S1132B6037720820F06000220921280000F012FBCF
S1132B7081481F210BA20A9BD2560A40012393408D
S1132B80036000BF08A20A9BD2560A400123934067
S1132B90036000BF05A20A9BD25611408C4004601A
S1132BA00BB0F0BD0E0000000E0000000E0038B5A2
S1132BB004002A4D696002216068A2689047606839
S1132BC0FFF716FF012061686854002032BD38B554
S1132BD004006068214D295C00290BD02249800043
S1132BE0085800F079FA00216068A2689047002034
S1132BF06168685431BD0000FFFFFFBFFFFF7FFF26
S1132C00F1B584B0170000240D00164E3000443096
S1132C10029014E00820029908600834FA20800029
S1132C2001900095029803893200403209210498EA
S1132C304068C0B200F022F8029800682D18BC4227
S1132C4006D2381B0928E5D2029908603C00E5E762
S1132C50002005B0F0BD0000FFEFFFFF54F2FF1F9E
S1132C60E129000030F1FF1F102F000010F0FF1FBA
S1132C70FF070000FFFF000021030000F0B585B04E
S1132C800D00914980000C58009990480840117833
S1132C9049058026B60331400143009100998C48D0
S1132CA0084051680904F02636030E400643009696
S1132CB00198400F400799042E4B0B4003430193A6
S1132CC000988449014000910A9900291AD00023F0
S1132CD00293039307E003980727FF1AFF00BE40FF
S1132CE0064303965B1CDBB2506883420AD2CE5C77
S1132CF0042BF0DA02980327FF1AFF00BE400643B4
S1132D000296EFE76A46E9B2200000F083FA002851
S1132D1014D10127AF40A06A3843A0626E4D0B9EC8
S1132D20310028000830FEF772F80328F8D0A16AB1
S1132D30B943A162002802D0052000E0012005B0BB
S1132D40F0BD000072A1800008582030016863497A
S1132D5001607047C529000048E8010020A1070070
S1132D6040420F0000B4C404206A5C48206270BD75
S1132D70F42E00000000FC1F00E100E0F1B586B075
S1132D8063A06946097E890040580090006B009951
S1132D90896A014001910198002847D04E4F386854
S1132DA00199C140C80735D538002030FEF766F8D0
S1132DB002AA3968C9B2009800F06AFA002829D139
S1132DC00026002402AD06E02C7B6846017E20002C
S1132DD07A6D9047761CF6B202980003000F864283
S1132DE018DA30000728F0D801A109568F4400BF33
S1132DF0080C1014181C20D8EC7AE6E7AC7AE4E747
S1132E006C7AE2E72C7AE0E7EC7BDEE7AC7BDCE78C
S1132E106C7BDAE778680199C140C80703D50837A5
S1132E203800FEF72BF80198009908630098006AAF
S1132E302A480099086207B0F0BD000070B506008A
S1132E4033A0B1004458206A61680A0405D54207DA
S1132E5003D53000FFF776FF70BD49042FD58107F5
S1132E602DD51F4DA978002928D0697801291FD1B3
S1132E701C4901400AD08C210902014006D10121DC
S1132E802000FFF770FD0020687017E02878401ECE
S1132E9040B2002800D50420287000BF15A00021EE
S1132EA069568A0051184118200000F03AF905E0EB
S1132EB02000FFF70FFD3000FFF79AFD54E721686B
S1132EC03000FFF75BFF70BD102F0000FFFFDFFF36
S1132ED0FFFFF0FFFFFFEFFF30F1FF1F02FC0000D8
S1132EE078F1FF1F0840000080B50020FFF7A6FF1F
S1132EF001BD0000070307070303030707030103DA
S1132F000707030103030305000305050700000089
S1132F1000400240802252030029016806D0490083
S1132F204908016001681140FCD1704780231B06E9
S1132F300B43036001681140FCD07047010000207E
S1132F408A4A914200D00120704701688022D2054C
S1132F500A4302600168802252050A430260016844
S1132F60C901FCD570470168814A0A4002600168C2
S1132F70804A0A4002600168C901FCD470470268B3
S1132F8092000AD5406B0001000F4200D21DD2B25C
S1132F908A428041C043C00F70470020704730B55B
S1132FA00168754A0A4002600168C902FCD48021A4
S1132FB0890402680A43026002680A40FCD101687D
S1132FC06E4A0A43026080214160B32109044163CF
S1132FD0002100226A4B88252D01940004196351B5
S1132FE0521C102AF9DB036143618361836400226C
S1132FF01301C31880331960521C102AF8DB30BD4A
S1133000F0B583B005000E001700FFF797FF00BF6F
S11330103DA180000858010C5A4A891801240A6805
S11330200123834013430B6000212800FFF772FF44
S113303030790028696802D15348084001E06003F0
S11330400843686001212800FFF764FF2800FFF7A8
S1133050A6FF29687F2081437079401E4006400EF8
S11330600843B17900296A6802D02103114301E0C1
S1133070654911406960F179002902D0A105014335
S113308001E062490140307A002802D0200408435C
S113309001E05F480840717A002902D0A10401438D
S11330A001E035490140296031680A20414300D1DB
S11330B001213800FDF718FD401EFF2800D9FF202C
S11330C069460870032088700220C8700C714C7027
S11330D0280000F026F8F7BD10B50400FFF75FFFE5
S11330E000212000FFF716FF2000FFF727FF8000D4
S11330F005A10858010C234A89180A680123834052
S11331009A430A6010BD000004003C1000210171C4
S11331105D4A0260102242718171C1710172417273
S1133120704738B505000C00FFF70FFF6868574972
S113313001406960686821780A0661788B05C021BE
S1133140090419401143A278D304E02292031A40DF
S11331500A43E1780904E023DB020B40134321799D
S11331604907490F1943014369600FE000400240D9
S1133170FFFFFFEFFFFFFFBFFFFFFBFF0F00280074
S1133180FFFFFF3F00700440FFDFFFFF2800FFF751
S1133190EAFE31BD70B504000D001600FFF7EFFE26
S11331A02801201880300021002E03D0802212052F
S11331B0026000E0016041608160C16070BDF2B5F1
S11331C0040016001F000025FFF7D9FE68460078AA
S11331D0000120188030056045608560C560002FBF
S11331E011D0316841603179012901D18025AD03C5
S11331F07179012903D1290080256D030D438021B4
S1133200C90429430160F1BDFFEFFFFFFFFFBFFFCA
S1133210FFFFFEFFF8B504000F0016000025FFF7BE
S1133220AEFE380120188030C02109050268F02361
S11332301B0513408B4224D00268314B134080227B
S113324012051A4302607268D200D20842603268E2
S11332500123540D1C4000D04D09140D234003D00C
S11332602B0080256D031D43F0231B0313401943DA
S113327029430D00B1688160F168C16005600020D8
S1133280F2BD0120F2BD000048E80100F8FF000093
S1133290F8B504000E001500FFF771FE3001201888
S11332A0803001680A01120F022A01D0062A24D1B3
S11332B04368DB00DB086E68760F760733436B6088
S11332C02E68104B33408E02F70F7E051E430E4BC3
S11332D03340CE02F70F3E051E43F0231B030B4081
S11332E033432B608168A960C068E860A068022A43
S11332F001D10020F2BD0548F2BDA0680120F2BD55
S1133300FFFFFFF0FFFFDFFFFFFFE0FFB914000046
S1133310010C114A89180A680123834013430B6086
S11333207047010C0C4A89180A68012383409A43A8
S11333300A6070470029817803D080220A43827092
S113334070474906490E8170704701000020034A06
S1133350914200D001207047007004400060064094
S11333604022114202D083781A43827020221140F5
S113337002D081790A43827170470100C8788A7942
S1133380520603D502008020C00110438979C90682
S113339003D50100802040010843704738B505007B
S11333A00C00FFF7D2FF264980000858FFF7B0FF52
S11333B0A07A002802D0022804D00DE0E088400062
S11333C0287009E0E0884000287020894000E871F6
S11333D06879082101436971A878FD210140A0782A
S11333E0400008432178C9010143A97068796F211D
S11333F001402079000108436178C9010143DF20BD
S11334000840E17849010143697131BD10B500BF3D
S113341004000021FFF78EFF2000FFF796FF00BF96
S113342008A180000858FFF77CFF10BD00218172BD
S113343041708170C17001710121017070470000F9
S11334404434000006003410002100BF04A28B00A5
S1133450D358834202D0491C0229F8D3080070478C
S113346000A0064000B00640FEB504000E001700A0
S1133470306800900001029038000299FDF734FB97
S113348085B2002D00D1012578010299FDF72CFBAE
S11334906901401A01907800019A92B28918FDF7E7
S11334A023FB0099471A08466421FDF71DFB4100E0
S11334B00818B84201D24948FEBD2000FFF7C4FFF6
S11334C02FA180000858010C454A89180A68012375
S11334D0834013430B60E078F3210140E170E02066
S11334E0217801402A120A4322706570A17A0840AB
S11334F00199C906C90E0143A172A078EC210140CB
S113350030790843A0702078DF21014070794001B0
S11335102022104008432070B079E074F07960757F
S1133520207C882101432174607CC02101436174A3
S1133530E078317A002902D0010008200843717A2A
S1133540002902D0010004200843E0700020FEBDE1
S113355080B5017D0029FCD101794906FCD5002103
S1133560C170FFF771FF800005A10858010C1C4AC7
S113357089180A68012383409A430A6001BD000048
S11335800A0034100B003410E121490201600021CB
S11335900171417181710122C271017241727047DE
S11335A002780B0013430370C2780B0A1343C370F1
S11335B082790B0C13438371427C090E11434174CD
S11335C0704705E003791B06FCD50B78C371491CD1
S11335D013005A1E002BF5D170470000F5030000BC
S11335E0007004400029817803D080220A4382704D
S11335F070474906490E8170704738B5694C200000
S1133600FFF7BBFE12220240E27050210140102954
S113361012D01021644AEF23450612D54007A07842
S11336200BD50143A1700020694608706846D16833
S1133630884768460078207131BD0340A370207923
S113364031BDA5780D4203D0C007ECD5A078F4E7CE
S1133650207900211269904731BD53494068085CC4
S1133660704751498A68002A08D04A681378037061
S1133670521C4A608868401E8860704700210170AF
S1133680704780B548494969884701BD5A2800D028
S1133690704780B5444A0123535444491161516928
S11336A0884701BDF0B585B004003F4E7161022129
S11336B06068A26890476068009000BF3FA00099CE
S11336C08900455801A8FFF7B1FE01A81021C18067
S11336D037498968096979310978FF2900D0C1809F
S11336E001A92800FFF75AFE01212800FFF77AFFFD
S11336F040212800FFF734FEFEF762FD2F00FA2177
S11337008900FDF7F1F901002A48FDF7EDF90021E0
S113371000E011004A1C13004343322BF9D3012566
S1133720002905D1FF22F632904204D2012102E0A1
S1133730202900D31F21B879F02202401143B97126
S113374001210098FEF7F6FE1B48306160683018CE
S11337504570002005B0F0BD70B504006068124DDE
S113376029184978002914D014A182008E58002108
S1133770FEF7E0FE00213000FFF734FF3000FFF7D2
S113378045FE00216068A2689047002061686918BE
S1133790487070BD04484160826081680029FCD192
S11337A0002070470060064088F0FF1F8336000049
S11337B010F0FF1F40420F008D36000000600640ED
S11337C010B5964880680469683434219448FEF73B
S11337D045FE002808D1342291492000FDF78CFBD6
S11337E020689049884204D0FF2234212000FDF74C
S11337F079FEFEF719FD002010BDF8B5874DA868C5
S113380004694B20E0700220A070002666702670C8
S11338105021E1710127A771607126715420E07273
S1133820A7726672267227637F4860632200103293
S11338300421280020302B69DB6A984722001432C7
S11338400121280020302B69DB6A984722001832B6
S11338500021280020302B69DB6A984722001C32A3
S11338600221280020302B69DB6A9847220020328D
S11338700321280020302B69DB6A98472200443258
S11338800521280020302B69DB6A98472200483242
S11338900621280020302B69DB6A984722004C322D
S11338A00721280020302B69DB6A9847A169484228
S11338B00021C9435D4A53420340C91A5C4A10407F
S11338C0A065E1655B4820665B4860666869E66000
S11338D007E07822A35C0B4202D0E2681143E16066
S11338E0761C1821714341580029F2D153480168CC
S11338F021644168E1638068A063686810300168EE
S1133900616241680068081A401CA0622000FDF74B
S113391023F927650020F2BDF8B517001E003F4AC1
S1133920916809690424464D401E172850D801A304
S11339301B5C9F4416262A2E323642469A4A4E5C17
S11339409A3A3E626880868A8E929A96002E00D0B9
S11339503460002F00D039600020F2BD0C31F5E74F
S11339601031F3E71431F1E71831EFE72031EDE7D7
S11339702431EBE72831E9E73431E7E72C31E5E797
S11339803031E3E7D06941694969884728602900F3
S1133990DCE710245831D9E72A480068F6E769467D
S11339A01000203012699269904768460078002818
S11339B0ECD00120EAE70C243831C7E74431C5E7ED
S11339C04831C3E74C31C1E75031BFE70831BDE7A7
S11339D01D48F2BD02001148806803691B48521E4D
S11339E0072A17D9093A0AD0521E012A12D9D21E1F
S11339F0032A0FD9083A08D0921E0BD00CE00029F4
S1133A0001D0012909D1196302E0032905D21965FE
S1133A1000207047401E7047801E704710F0FF1F43
S1133A20C0A300006B6366677F0D00007041000057
S1133A300000000000F0FF1FCFF5FF1F5880044076
S1133A4030F3FF1F248004403C2800003E2800007F
S1133A5010B50100A34A1000883003685C1C0460A0
S1133A60D2182032117001688906890E016010BDD8
S1133A700020704780B500F0C6F802BDFAB583B0E7
S1133A801700002901D0002F01D104202CE00026CA
S1133A903E60944C200090300090467000F0B3F8E3
S1133AA0002821D101AD02E0A22000F082F82021FB
S1133AB02000FDF737FD6846027C210001A800F0D4
S1133AC013F9002801D03E600EE0210001A800F0A7
S1133AD089F9A9888142E7D10120009908700398E7
S1133AE0046068883860002005B0F0BDF2B582B08B
S1133AF015001F00002944D0212D42D200F083F884
S1133B0000284DD1774C20009130002601780029FF
S1133B1000D006702000603000905A200099087090
S1133B20A42000994870002F02D0A5200099487065
S1133B30200062300570290A4170002D05D02A004A
S1133B40029920006630FDF7C3F921006631009820
S1133B5000F048F964342070000A6070A91D0098D0
S1133B6000F064F800281BD101AC01A800F028F98A
S1133B70002815D16078A12811D0A22805D0A32847
S1133B8001D00420FEBD8848FEBD00984188891DEF
S1133B9000F04CF8002803D16078A228E5D000207A
S1133BA0FEBD8248012181700021017070472020F0
S1133BB0704780B569465A220A70487001207C49D2
S1133BC008700221684600F031F802BD10B582B0D9
S1133BD004007648017842780A408078024210D185
S1133BE0684600BF8DA10A8802800222694620002F
S1133BF023695B689847082289A1200023695B68D0
S1133C0098476C4816BD80B5684800210278002AA0
S1133C1002D00170A12004E08278002A04D08170CF
S1133C20A320FFF7C6FF02BD002002BD80B503003C
S1133C306148C0690A00190003695B68984702BDBE
S1133C40F3B585B015000024FCF721FE6A4603C2D3
S1133C50FA20800045432800FCF729FE02AA03C28B
S1133C60564D0FE06868296888420ED01D4908182F
S1133C702030007805990855641C6868401C80064B
S1133C80800E68600698844229D0FCF700FE02008A
S1133C900B00684603C81F00161A8F41684603C804
S1133CA08B420DD801D382420AD2684603C8C0436E
S1133CB0C94312184B410020521C434116001F00F7
S1133CC002A803C8002901D10028CBD002A803C848
S1133CD08F42C7D301D88642C4D3052000E0002018
S1133CE007B0F0BD34F3FF1F70B582B004000D00BF
S1133CF0160000F065F8002855D16078A62804D194
S1133D002D48C069FFF762FF76BDA421002E00D0C4
S1133D10A521884201D0012076BD142202216846E3
S1133D20FFF78EFF69460988A170090AE17000282F
S1133D3039D1A078E1780906090C0843212801DB70
S1133D40202004E0A078E1780906090C0843A0705B
S1133D50000AE070142202216846FFF771FF6946E9
S1133D6009882171090A617100281CD1A178E278BF
S1133D701206120C114316D0A178E0780006000C4C
S1133D8001432800FDF7CCFBA078E1780906090C73
S1133D900843A178E2781206120C11430A22424326
S1133DA02800FFF74DFF76BD12270000C4F3FF1F64
S1133DB0C5F3FF1F1327000010F0FF1FBCF3FF1F04
S1133DC010B50400002201212000FFF739FF00286C
S1133DD007D120785A28F5D10A220121601CFFF767
S1133DE02FFF10BD30B583B004000D006846FEF708
S1133DF0C7FB042221006846FEF7C5FBA278E078E1
S1133E000006000C024329006846FEF7BCFB01A92A
S1133E106846FEF7E1FB684680883EBD5AA700006D
S1133E20000201500000AAEA00480047293E0000B1
S1133E3004480549C1810549C181E921490001803E
S1133E40704700BF0020054020C5000028D90000AD
S1133E507FB5040069466068FCF78AFC002831D10C
S1133E606068012801D0394D00E0394D01A8FFF701
S1133E708BFB00980190012601A8067246726068C7
S1133E80FEF7AAF9020001A92800FFF7EDFA0028BD
S1133E9015D101216068FEF75DFB71032800FFF76F
S1133EA07FFB02216068A26890472A4C5A2061680F
S1133EB08847A620616888472670012003E060686F
S1133EC0FCF73CFC002004B070BD10B50400214890
S1133ED0416001216068A26890476068FCF72EFC8D
S1133EE0002010BD10B504001A48007800280BD03B
S1133EF000216068FEF72EFB6068012801D013489A
S1133F0000E01348FFF724FB00216068A268904793
S1133F1010BD80B54068012801D00C4800E00C4871
S1133F20FFF74FFB002002BD0B480178890600D43F
S1133F30704780B505E009480178890600D47047C8
S1133F4080B5C07803494968884701BD00A0064090
S1133F5000B00640C8F3FF1F04A0064004B00640AA
S1133F6000F00BF8002801D000F00AF80020C04649
S1133F70C046FDF782FDFDF79FFD0120704700005C
S1133F8010B5074979441831064C7C44163404E0D2
S1133F90081D0A68891888470100A142F8D110BD9C
S1133FA0C0010000CC010000990F0000A50F000023
S1133FB0EC04000090F1FF1F4C060000A0F0FF1F6E
S1133FC0F406000000F0FF1F7C0500007C060000E2
S1133FD000000000000000000000000000000000DD
S1133FE000000000000000000000000000000000CD
S1133FF000000000000000000000000000000000BD
S113400000000000000000000000000000000000AC
S1134010C8F1FF1F08F2FF1F0000000000000000AD
S1134020000000000126000021260000000000001E
S113403000000000000000000000000063360000E3
S11340408D3600000000000000000000FFFF0100AA
S1134050010000000406000000F0FF1FFF2F0020F5
S1134060010000006406000000000040FFFF07405C
S113407000000000D405000000F00F40FFFF0F40D7
S113408000000000D4050000000000E0FFFF0FE086
S113409000000000D4050000000000000000000043
S11340A000000000000000000000400130B504E002
S11340B014780470401C521C491E002919D0C507ED
S11340C0F6D40129F4D0850701D4042904D2148834
S11340D00480801C921C891E8B08EED09B00C4189F
S11340E003E015680560001D121DA042F9D3C91A2A
S11340F0E3E730BD80B513000200180000E080B58E
S1134100FFF7D4FF002002BD10B50C0011000123FD
S11341102200FCF7ADF910BDC046C046C046C046FB
S1134120FFF71EFF70B40121002313E00468001D93
S11341300C4202D04D466D1E64192360241D121FCB
S1134140042AFAD22500960701D52380AD1C0A4023
S113415000D02B700268001D002AE7D170BC7047A4
S1134160C5FFFFFFC802000008F1FF1F00000000A8
S9030411E7
